:100000002DEF15F0FFFFFFFF00C06DF3E9CFC3F246
:10001000EACFC4F2E1CFC5F2E2CFC6F2C20ED76E8C
:10002000F70ED66E200EF26E837E152A3C0E155CFE
:1000300003E3010E166E156AC3C2E9FFC4C2EAFFEC
:10004000C5C2E1FFC6C2E2FF6DC300F0110017C0D8
:10005000E9FF18C0EAFF1950EF166CC3C9FFC7A02B
:10006000FED71A50EF12C9CF00F01200FF0E0301A5
:100070006C6F27EC00F0400E030163256C6F27ECDA
:1000800000F067C36CF327EC00F066C36CF327EC59
:1000900000F065C36CF327EC00F064C36CF327EC4D
:1000A00000F068C36CF327EC00F0FF0E03016C6FE7
:1000B00027EC00F000C069F303016A6B6B6B03016E
:1000C0006951000A17E06951010A14E06AC301F09E
:1000D0006BC302F06A4B6B2B4E0E025C02E1200EEA
:1000E000015C08E2FF0E03016C6F27EC00F000C01A
:1000F00069F3E5D769C300F01200090E006E59C319
:1001000064F35AC365F35BC366F35CC367F30050E3
:1001100008E0030164376491653766376737FF0F7E
:10012000F7D7110E0301636FFF0E686F36EC00F016
:10013000005203E0010E006E1200FF0E03016C6F0F
:1001400027EC00F00050FE0AF8E103015F6B606BE2
:10015000020E0301605D02E1000E5F5D15E2030126
:100160005F515D25616F60515E21626FFF0E6C6FA4
:1001700027EC00F061C3E1FF62C3E2FF00C0E6FFCD
:1001800003015F4B602BE4D7FF0E03016C6F27EC7C
:1001900000F0FF0E03016C6F27EC00F0006A120004
:1001A000090E006E59C364F35AC365F35BC366F36B
:1001B0005CC367F3005008E003016437649165375E
:1001C00066376737FF0FF7D7180E0301636FFF0E0F
:1001D000686F36EC00F0005203E0010E006E120072
:1001E000FF0E03016C6F27EC00F0FF0E03016C6F34
:1001F00027EC00F0FE0E03016C6F27EC00F003010A
:100200005F6B606B03016051010802E15F51FF0801
:100210000FE303015F515D25E96E60515E21EA6ED7
:10022000EECF6CF327EC00F003015F4B602BEAD7B5
:10023000FF0E03016C6F27EC00F0FF0E03016C6FE3
:1002400027EC00F0FF0E03016C6F27EC00F000C0FC
:100250005FF3000E0301606F1F0E5F15016E60C338
:1002600002F0000E021601C05FF302C060F3000E40
:10027000021802E1050E011803E0020E006E1200E2
:10028000FF0E03016C6F27EC00F00050FF0AF8E14D
:10029000006A120000010B6A0A6A096A005004022F
:1002A000F4CF09F0F3CF08F001500502F4CF0BF0C2
:1002B000F3CF0AF000500502F3500926F4500A2249
:1002C000E86A0B2201500402F3500926F4500A2276
:1002D000E86A0B2208C000F009C001F00AC002F071
:1002E0000BC003F0120003015951390807E3300E27
:1002F000595D04E3010E006E7FEF01F0006A120009
:10030000000100500402F4CF09F0F3CF08F00150CF
:100310000502F4CF0BF0F3CF0AF000500502F350C2
:100320000926F4500A22E86A0B2201500402F35015
:100330000926F4500A22E86A0B2205AEA4EF01F068
:1003400000500A5C01500B5801AEABEF01F00450B5
:100350000A5C05500B5808C000F009C001F00AC043
:1003600002F00BC003F012000001086A096A100EC7
:100370000C6E0134083609360450085E0550D8A0CA
:10038000053C095ED8B0CCEF01F0045008260550BA
:10039000D8B0053C0926D890003601360C2EB9EFAE
:1003A00001F0120000001200080E0B6EFF0E0A6E24
:1003B0000B2E01D003D00A2EFED7FAD71E0E0A6EDE
:1003C0000A2EFED71200100E0A6E0A2EFED700006B
:1003D000120000010B6A0A6A096A086A0E6A03348D
:1003E00008360450085E0550D8A0053C095E06504A
:1003F000D8A0063C0A5E0750D8A0073C0B5EE86A0E
:10040000D8A0010E0E5E0336070E0C6E03340836BC
:1004100009360A360B360E36045003A023EF02F0DD
:10042000085E0550D8A0053C095E0650D8A0063CE1
:100430000A5E0750D8A0073C0B5EE86AD8A0010E00
:100440000E5E34EF02F008260550D8B0053C0926B0
:100450000650D8B0063C0A260750D8B0073C0B26F9
:10046000E86AD8B0010E0E2603360C2E06EF02F015
:100470000234083609360A360B360E36045003A00D
:1004800055EF02F0085E0550D8A0053C095E065005
:10049000D8A0063C0A5E0750D8A0073C0B5EE86A6D
:1004A000D8A0010E0E5E66EF02F008260550D8B007
:1004B000053C09260650D8B0063C0A260750D8B09D
:1004C000073C0B26E86AD8B0010E0E260236070E4E
:1004D0000C6E0234083609360A360B360E360450D6
:1004E00002A086EF02F0085E0550D8A0053C095E28
:1004F0000650D8A0063C0A5E0750D8A0073C0B5E09
:10050000E86AD8A0010E0E5E97EF02F008260550AB
:10051000D8B0053C09260650D8B0063C0A2607503C
:10052000D8B0073C0B26E86AD8B0010E0E2602367A
:100530000C2E69EF02F00134083609360A360B3604
:100540000E36045002A0B8EF02F0085E0550D8A0A5
:10055000053C095E0650D8A0063C0A5E0750D8A0AC
:10056000073C0B5EE86AD8A0010E0E5EC9EF02F0F0
:1005700008260550D8B0053C09260650D8B0063CE0
:100580000A260750D8B0073C0B26E86AD8B0010EFF
:100590000E260136070E0C6E0134083609360A366F
:1005A0000B360E36045001A0E9EF02F0085E05504C
:1005B000D8A0053C095E0650D8A0063C0A5E07504C
:1005C000D8A0073C0B5EE86AD8A0010E0E5EFAEFD9
:1005D00002F008260550D8B0053C09260650D8B0D0
:1005E000063C0A260750D8B0073C0B26E86AD8B06C
:1005F000010E0E2601360C2ECCEF02F00034083628
:1006000009360A360B360E36045001A01BEF03F0F4
:10061000085E0550D8A0053C095E0650D8A0063CEF
:100620000A5E0750D8A0073C0B5EE86AD8A0010E0E
:100630000E5E2CEF03F008260550D8B0053C0926C5
:100640000650D8B0063C0A260750D8B0073C0B2607
:10065000E86AD8B0010E0E260036070E0C6E003484
:10066000083609360A360B360E36045000A04CEF19
:1006700003F0085E0550D8A0053C095E0650D8A0DE
:10068000063C0A5E0750D8A0073C0B5EE86AD8A07B
:10069000010E0E5E5DEF03F008260550D8B0053C54
:1006A00009260650D8B0063C0A260750D8B0073CA9
:1006B0000B26E86AD8B0010E0E2600360C2E2FEF5E
:1006C00003F000B072EF03F0045008260550D8B0D4
:1006D000053C09260650D8B0063C0A260750D8B07B
:1006E000073C0B26120003011A6B1B6A1C6A040EDE
:1006F0001D6E000E1E6E1FC059F320C05AF321C09C
:100700005BF322C05CF3230E5D6F000E5E6F7DEC29
:1007100000F01E500201241902E123511D1817E1B7
:100720001D6A1E6A1B4A1C2A1B501F240301596F95
:100730001C5020205A6F000E21205B6F000E2220DB
:100740005C6F230E5D6F000E5E6F7DEC00F0230E7C
:100750001D24E96E000E1E20EA6EEECF02F002505C
:10076000000A14E1010E1D24006E000E1E20016E11
:10077000230E0024E96E000E0120EA6EEECF02F097
:100780000250000A03E1010E03011A6F020E1D263A
:10079000000E1E2203011A53BCE003011A6B020E65
:1007A0001D5E000E1E5A1200230E1D24E16E000E67
:1007B0001E20E26EFF0EE66E010E1D24006E000E7E
:1007C0001E20016E230E0024E16E000E0120E26E59
:1007D000FF0EE66E1B501F240301596F1C50202092
:1007E0005A6F000E21205B6F000E22205C6F230EDB
:1007F0005D6F000E5E6FD0EC00F01B5002012525EE
:100800000301596F1C500201262103015A6F000E8B
:100810000201272103015B6F000E02012821030161
:100820005C6F230E5D6F000E5E6FD0EC00F0120067
:100830001BC000F01CC001F02BC204F02CC205F05C
:100840004AEC01F01DC002F01EC003F00332023278
:10085000039E025000240201296F035001202A6FD9
:100860001200020E0201295D006E000E2A59016E6F
:1008700031C204F0000E056E4AEC01F000C02DF20A
:1008800001C02EF2000E02012F6F306F32512D2762
:1008900033512E2334512F23355130231200070EAC
:1008A0000A6E0A2EFED712006E0E0301216F6F0E24
:1008B000226F6E0E236F2D0E246F6C0E256F6F0E40
:1008C000266F6E0E276F670E286F200E296F700E31
:1008D0002A6F720E2B6F690E2C6F6E0E2D6F740EB9
:1008E0002E6F660E2F6F306B6E0E316F6F0E326F84
:1008F0006E0E336F2D0E346F660E356F6C0E366FC5
:100900006F0E376F610E386F740E396F200E3A6FAD
:10091000700E3B6F720E3C6F690E3D6F6E0E3E6F38
:10092000740E3F6F660E406F416B280E426F6E0E65
:10093000436F750E446F6C0E456F6C0E466F290E3B
:10094000476F486B506B516B4E6B4F6B1CC300F085
:100950001DC301F01EC302F0010E03011C27000E8F
:100960001D231E2300C0F6FF01C0F7FF02C0F8FFE1
:100970000900F5CF00F000C04BF30052D8B4BCEF33
:100980000BF04B51250A0BE01AC3E1FF1BC3E2FF3A
:100990004BC3E6FF1A4B1B2B504B512BD7D70301F0
:1009A0004C6B4D6B4E6B4F6B28D003014E87010E85
:1009B0001C27000E1D231E235ED003014E81010E55
:1009C0001C27000E1D231E2356D003014E83010E4B
:1009D0001C27000E1D231E234ED003014F87010E3E
:1009E0001C27000E1D231E2346D003014E85010E39
:1009F0001C27000E1D231E233ED01CC3F6FF1DC363
:100A0000F7FF1EC3F8FF0900F5CF56F30301565157
:100A10002D0ACBE01CC3F6FF1DC3F7FF1EC3F8FF72
:100A20000900F5CF56F35651200AC7E01CC3F6FF64
:100A30001DC3F7FF1EC3F8FF0900F5CF56F356514B
:100A40002B0AC3E01CC3F6FF1DC3F7FF1EC3F8FF4C
:100A50000900F5CF56F35651230ABFE01CC3F6FF39
:100A60001DC3F7FF1EC3F8FF0900F5CF56F356511B
:100A7000300ABBE001D098D703014EB34E91030179
:100A80004EB74E951CC3F6FF1DC3F7FF1EC3F8FFFC
:100A90000900F5CF00F0000E016E00C059F373ECB1
:100AA00001F0005238E003014C6B4D6B4CC300F079
:100AB0004DC301F00A0E046E000E056E80EC01F0CD
:100AC0001CC3F6FF1DC3F7FF1EC3F8FF0900F5CFD7
:100AD00056F30301565100244C6F000E01204D6F58
:100AE000300E4C5F000E4D5B010E1C27000E1D23C7
:100AF0001E231CC3F6FF1DC3F7FF1EC3F8FF09002A
:100B0000F5CF00F0000E016E00C059F373EC01F058
:100B10000052CCE136D01CC3F6FF1DC3F7FF1EC345
:100B2000F8FF0900F5CF56F3030156512A0A29E1CF
:100B30001FC3E9FF20C3EAFFEECF00F0EECF01F0C4
:100B400000C0E9FF01C0EAFFEECF4CF3EECF4DF35A
:100B50001FC3E9FF20C3EAFFEECF00F0EECF01F0A4
:100B6000020E0026000E01221FC3E1FF20C3E2FF98
:100B700000C0E6FF01C0E6FF010E1C27000E1D238A
:100B80001E231CC3F6FF1DC3F7FF1EC3F8FF090099
:100B9000F5CF56F3030156512E0A75E1010E1C27BD
:100BA000000E1D231E231CC3F6FF1DC3F7FF1EC32B
:100BB000F8FF0900F5CF56F356512A0A2AE11FC360
:100BC000E9FF20C3EAFFEECF00F0EECF01F000C056
:100BD000E9FF01C0EAFFEECF49F3EECF4AF31FC3AE
:100BE000E9FF20C3EAFFEECF00F0EECF01F0020EE6
:100BF0000026000E01221FC3E1FF20C3E2FF00C058
:100C0000E6FF01C0E6FF010E1C27000E1D231E2378
:100C100038D00301496B4A6B1CC3F6FF1DC3F7FFB5
:100C20001EC3F8FF0900F5CF00F0000E016E00C0F2
:100C300059F373EC01F0005224E049C300F04AC3B9
:100C400001F00A0E046E000E056E80EC01F01CC36C
:100C5000F6FF1DC3F7FF1EC3F8FF0900F5CF56F3DB
:100C6000030156510024496F000E01204A6F300ED7
:100C7000495F000E4A5B010E1C27000E1D231E2338
:100C8000CBD7030103D00301496B4A6B1CC300F0AF
:100C90001DC301F01EC302F0010E03011C27000E4C
:100CA0001D231E2300C0F6FF01C0F7FF02C0F8FF9E
:100CB0000900F5CF4BF313D150C300F051C301F03D
:100CC0001200210E0301526F030E536F496B4A6BE2
:100CD000FF0E4E6FFF0E4F6F35D0310E0301526F76
:100CE000030E536F496B4A6B2DD003014E8D33D1E8
:100CF00032D103014E8B03014E8F2DD11FC3E9FF6B
:100D000020C3EAFFEECF00F0EECF01F000C0E9FF14
:100D100001C0EAFFEECF52F3EECF53F31FC3E9FF5A
:100D200020C3EAFFEECF00F0EECF01F0020E002666
:100D3000000E01221FC3E1FF20C3E2FF00C0E6FF57
:100D400001C0E6FF000E0301531902E1000E521923
:100D500005E1420E0301526F030E536F0301546B02
:100D6000556B030154515225E96E55515321EA6EDA
:100D7000EECF00F0005203E0544B552BF2D70301A5
:100D800049514A110AE055514A5D02E15451495D09
:100D900004E249C354F34AC355F303014D51555D71
:100DA00002E14C51545D06E2030154514C5F555130
:100DB0004D5B03D003014C6B4D6B03014EB717D055
:100DC0004CC300F04DC301F0010E03014C5F000E57
:100DD0004D5B005001100BE01AC3E1FF1BC3E2FFA3
:100DE000200EE66E1A4B1B2B504B512BE9D754C3E8
:100DF00000F055C301F0010E0301545F000E555B76
:100E00000050011013E052C3E9FF53C3EAFFEECFD5
:100E100000F01AC3E1FF1BC3E2FF00C0E6FF1A4B5C
:100E20001B2B524B532B504B512BE1D703014EA799
:100E300017D04CC300F04DC301F0010E03014C5F0D
:100E4000000E4D5B005001100BE01AC3E1FF1BC305
:100E5000E2FF200EE66E1A4B1B2B504B512BE9D7AD
:100E600003014F51FF0A02E1FF0E4E1905E150C385
:100E700000F051C301F0120069D51FC3E9FF20C380
:100E8000EAFFEECF00F0EECF01F000C0E9FF01C0B5
:100E9000EAFFEECF4BF31FC3E9FF20C3EAFFEECF1B
:100EA00000F0EECF01F0020E0026000E01221FC35B
:100EB000E1FF20C3E2FF00C0E6FF01C0E6FF4B0EEA
:100EC0000301526F030E536F010E546F000E556FE6
:100ED00056D7C00E03014E13000E4F133CD0030132
:100EE0004B51000AD8B4E8D64B516C0AD8B4E9D6B5
:100EF0004B51450AD8B4F1D64B51660AD8B4EDD659
:100F00004B51650AD8B4E9D64B51670AD8B4E5D637
:100F10004B516F0AD8B4E9D64B51640AD8B4E8D61D
:100F20004B51690AD8B4E4D64B51700AD8B4E1D613
:100F30004B51580AD8B4DDD64B51780AD8B4DBD619
:100F40004B51730AD8B4DAD64B51630A96E04B5131
:100F5000750ABFE0B4D7C00E03014E15566F4FC3DC
:100F600057F3000E5717000E571902E1000E5619DD
:100F70003FE11FC3E9FF20C3EAFFEECF00F0EECF51
:100F800001F000C0E9FF01C0EAFFEECF52F3EECF5F
:100F900053F31FC3E9FF20C3EAFFEECF00F0EECF0B
:100FA00001F0020E0026000E01221FC3E1FF20C344
:100FB000E2FF00C0E6FF01C0E6FF800E0301531907
:100FC000006E800E005C02E1000E525D10E2030E26
:100FD00003014E13000E4F1352510008006E53C30D
:100FE00001F0E86A015600C052F301C053F324D067
:100FF0001FC3E9FF20C3EAFFEECF00F0EECF01F000
:1010000000C0E9FF01C0EAFFEECF52F3EECF53F389
:101010001FC3E9FF20C3EAFFEECF00F0EECF01F0DF
:10102000020E0026000E01221FC3E1FF20C3E2FFD3
:1010300000C0E6FF01C0E6FF000E03014A1902E10D
:10104000000E49190AE1000E0301531902E1000ED6
:10105000521903E10301494B4A2BC00E03014E15FF
:10106000006E00C058F39FD0010E03014B6F0301C7
:101070004B51050A2DE0010E046E4BC300F0000E2B
:10108000016E026E036E045007E0003600900136D8
:1010900002360336FF0FF8D73A0E00262D0E012236
:1010A000000E022200C0F6FF01C0F7FF02C0F8FFE9
:1010B0000900F5CF56F30900F5CF57F30301575157
:1010C000535D02E15651525D03E303014B2BCFD731
:1010D00079D0010E03014B6F03014B51040A2DE03F
:1010E000010E046E4BC300F0000E016E026E036E23
:1010F000045007E000360090013602360336FF0F39
:10110000F8D7440E00262D0E0122000E022200C048
:10111000F6FF01C0F7FF02C0F8FF0900F5CF56F354
:101120000900F5CF57F303015751535D02E15651C2
:10113000525D03E303014B2BCFD744D0010E0301D3
:101140004B6F03014B51060A2DE0010E046E4BC399
:1011500000F0000E016E026E036E045007E00036D0
:101160000090013602360336FF0FF8D74C0E0026EA
:101170002D0E0122000E022200C0F6FF01C0F7FF73
:1011800002C0F8FF0900F5CF56F30900F5CF57F379
:1011900003015751535D02E15651525D03E30301D0
:1011A0004B2BCFD70FD003015851000AD8B45CD7CE
:1011B0005851C00AD8B458D75851800A8AE05851BB
:1011C000400ABCE0800E006E800E03014A19005CEC
:1011D00002E149514B5D03E249C34BF30FD0800E4E
:1011E00003014A19006E800E005C02E14B51495D1B
:1011F00005E24BC349F3000E03014A6F03014C5152
:101200004D110FE0030E4E15006E4FC301F0000E9E
:1012100001160050011005E0010E03014C5F000EA5
:101220004D5B800E03014A19006E800E4D19005C63
:1012300002E14C51495D06E2030149514C5F4A51BC
:101240004D5B03D003014C6B4D6BC40E03014E1577
:10125000566F4F51080B576F5751080A02E1400E65
:10126000561909E103014C514D1104E0010E4C5F88
:10127000000E4D5B20D0C00E03014E15566F4F512E
:10128000080B576F5751080A02E1800E561913E1F7
:10129000800E006E800E03014D19005C02E14C517E
:1012A000020806E2020E03014C5F000E4D5B03D004
:1012B00003014C6B4D6B03014EA574D04EA31BD0A4
:1012C000010E4E15006E4FC301F0000E01160050C6
:1012D000011003E02D0E006E02D02B0E006E1AC31B
:1012E000E1FF1BC3E2FF00C0E6FF03011A4B1B2B0B
:1012F000504B512B40D0010E03014E15006E4FC3D1
:1013000001F0000E0116005001100BE01AC3E1FFBE
:101310001BC3E2FF200EE66E1A4B1B2B504B512BCA
:101320002AD0C00E03014E15566F4F51080B576F50
:101330005751080A02E1800E56191DE11AC3E1FF58
:101340001BC3E2FF300EE66E03011A4B1B2B504B02
:10135000512B4EAB03D0580E006E02D0780E006EAB
:101360001AC3E1FF1BC3E2FF00C0E6FF03011A4BF3
:101370001B2B504B512B03014C514D1112E01AC342
:10138000E1FF1BC3E2FF300EE66E03011A4B1B2B7D
:10139000504B512B010E4C5F000E4D5B4C514D11CB
:1013A000EEE18ED003014C514D1114E04EB712D036
:1013B0001AC3E1FF1BC3E2FF200EE66E03011A4BC6
:1013C0001B2B504B512B010E4C5F000E4D5B4C51B3
:1013D0004D11EEE103014EA31BD0010E4E15006E20
:1013E0004FC301F0000E01160050011003E02D0E56
:1013F000006E02D02B0E006E1AC3E1FF1BC3E2FF8A
:1014000000C0E6FF03011A4B1B2B504B512B15D08C
:10141000010E03014E15006E4FC301F0000E0116C0
:10142000005001100AE01AC3E1FF1BC3E2FF200EC7
:10143000E66E1A4B1B2B504B512BC00E03014E1561
:10144000566F4F51080B576F5751080A02E1400E73
:1014500056190CE11AC3E1FF1BC3E2FF300EE66E22
:1014600003011A4B1B2B504B512B2AD0C00E0301EA
:101470004E15566F4F51080B576F5751080A02E12E
:10148000800E56191DE11AC3E1FF1BC3E2FF300EA7
:10149000E66E03011A4B1B2B504B512B4EAB03D066
:1014A000580E006E02D0780E006E1AC3E1FF1BC307
:1014B000E2FF00C0E6FF03011A4B1B2B504B512BE0
:1014C000800E006E800E03014A19005C02E1495152
:1014D0004B5D0CE21AC3E1FF1BC3E2FF300EE66E68
:1014E00003011A4B1B2B504B512BEAD749C300F079
:1014F0004AC301F0010E0301495F000E4A5B005030
:101500000110D8B419D1C00E4E15006E00C056F3AC
:10151000F7D0010E046E49C300F04AC301F0000E7B
:1015200003014ABFFF0E026E036E045007E000364F
:101530000090013602360336FF0FF8D73A0E002628
:101540002D0E0122000E022200C0F6FF01C0F7FF9F
:1015500002C0F8FF0900F5CF04F00900F5CF05F04F
:1015600052C300F053C301F0B4EC01F00A0E046E54
:10157000000E056EB4EC01F008C000F009C001F0E7
:10158000300E002403014B6FCBD04EAB42D0010E86
:10159000046E49C300F04AC301F0000E4ABFFF0EBB
:1015A000026E036E045007E00036009001360236EA
:1015B0000336FF0FF8D7440E00262D0E0122000E31
:1015C000022200C0F6FF01C0F7FF02C0F8FF0900C9
:1015D000F5CF04F00900F5CF05F052C300F053C376
:1015E00001F0B4EC01F00F0E0016000E0116000E13
:1015F000026E580E00262D0E0122000E022200C09F
:10160000F6FF01C0F7FF02C0F8FF0900F5CF4BF36A
:1016100042D0010E046E49C300F04AC301F0000E2F
:1016200003014ABFFF0E026E036E045007E000364E
:101630000090013602360336FF0FF8D7440E00261D
:101640002D0E0122000E022200C0F6FF01C0F7FF9E
:1016500002C0F8FF0900F5CF04F00900F5CF05F04E
:1016600052C300F053C301F0B4EC01F00F0E0016AA
:10167000000E0116000E026E6A0E00262D0E0122CB
:10168000000E022200C0F6FF01C0F7FF02C0F8FF03
:101690000900F5CF4BF344D0010E046E49C300F0AE
:1016A0004AC301F0000E03014ABFFF0E026E036E33
:1016B000045007E000360090013602360336FF0F73
:1016C000F8D74C0E00262D0E0122000E022200C07B
:1016D000F6FF01C0F7FF02C0F8FF0900F5CF04F0E4
:1016E0000900F5CF05F052C300F053C301F0B4EC8C
:1016F00001F0070E001403014B6F300E4B2710D082
:1017000003015651000AD8B404D75651C00AD8B4C0
:1017100000D75651800AD8B438D75651400ABCE099
:101720001AC3E1FF1BC3E2FF4BC3E6FF03011A4BE1
:101730001B2B504B512BDAD603014EA71BD0800E2A
:10174000006E800E4D19005C02E14C51000812E25F
:101750001AC3E1FF1BC3E2FF200EE66E03011A4B22
:101760001B2B504B512B010E4C5F000E4D5B4C510F
:101770004D11EEE1A6EF04F050C300F051C301F0AB
:10178000120002013651371100E036C2E9FF37C2BC
:10179000EAFF03011A5300E0EF96EF9EEF9CEF9AE9
:1017A000EF98EF941ABFEF8E1ABDEF8C1ABBEF8A39
:1017B0001AB9EF8802013851010A03E1EF94E2EF10
:1017C0000BF0EF84EF86D2EC01F003011A5300E036
:1017D000EF96EF9EEF9CEF9AEF98EF941AB7EF8E8B
:1017E0001AB5EF8C1AB3EF8A1AB1EF88020138519B
:1017F000010A03E1EF94FEEF0BF0EF84EF86D2ECE9
:1018000001F0EF9602013851010A03E1D4EC01F036
:1018100002D0E3EC01F01200A69C09C3A9FFA69E2A
:10182000A680A8CF00F01200A69CA6A202D00000BD
:10183000FCD709C3A9FF0AC3A8FFA69EA684F29EEF
:10184000550EA76EAA0EA76EA682F28EA69412005F
:101850000001086B080E0C6E003408360450085E58
:10186000D8B035EF0CF00826D89000360C2E2CEFAF
:101870000CF012000BC300F0010E016E005004E0EA
:1018800001360190FF0FFBD701C01AF0011C006E5A
:1018900000C019F0090E03010925176E000E0A2178
:1018A000186E17C0E9FF18C0EAFF0150EF12090EC9
:1018B0001724E96E0050EF16949A94889496210E9E
:1018C000C66E400EC76E0C6B0A0E03010C5D07E27C
:1018D000FF0E6C6F27EC00F003010C2BF5D7030112
:1018E000636B646B656B666B676B950E686F36EC4C
:1018F00000F00050010A02E0006A1200010E03012C
:10190000636F646B656B666B676BFF0E686F36ECBD
:1019100000F00052F3E1010E006E12000201396B7B
:101920003A6B3B6B3C6B3D6B3E6B3F6B406B416B73
:10193000426B436B446B296B2A6B2D6B2E6B2F6BA9
:10194000306B456B466B476B486B1F6A206A216A98
:10195000226A256B266B276B286B496B4A6B4B6B96
:101960004C6B1B6A1C6A4D6B4E6B1D6A1E6A4F6B7B
:10197000506B236B246B2B6B2C6B516B526B536B2B
:10198000546B556B566B326B336B346B356B316B01
:10199000576B586B596B5A6B5B6B5C6B5D6B5E6B1B
:1019A0005F6B606B616B120029C209F32AC20AF3F4
:1019B0000301093709910A37000E0B6F0C6F23C220
:1019C00004F024C205F0000E066E076E09C300F095
:1019D0000AC301F00BC302F00CC303F0E9EC01F001
:1019E00000C01BF001C01CF023C204F024C205F0AB
:1019F000000E066E076E09C300F00AC301F00BC3A8
:101A000002F00CC303F0E9EC01F008C000F009C0DB
:101A100001F00AC002F00BC003F000C01DF001C0CD
:101A20001EF0120002013F6B406B3D6B3E6B73EC8E
:101A300003F0D4EC03F018EC04F039C259F33AC2C5
:101A40005AF33BC25BF33CC25CF3230E03015D6FB0
:101A5000000E5E6F7DEC00F003010C6B0201405143
:101A6000241902E123513F191EE102013F6B406B33
:101A70003D4B3E2B3D5139250301596F02013E512B
:101A80003A2103015A6F000E02013B2103015B6FF3
:101A9000000E02013C2103015C6F230E5D6F000EFE
:101AA0005E6F7DEC00F0230E02013F25E96E000E13
:101AB0004021EA6EEECF02F00250E50A0BE0230E61
:101AC0003F25E96E000E4021EA6EEECF02F0025093
:101AD000000A03E1010E03010C6F200E02013F27F3
:101AE000000E402303010C53B9E003010C51010A1D
:101AF000D8A48FD0200E02013F5F000E405B03018F
:101B00000B6B03010B510A081BE30B5102013F252C
:101B1000006E000E4021016E230E0024E16E000EC7
:101B20000120E26E03010B510925E96E000E0A2126
:101B3000EA6EEECF00F000C0E6FF03010B2BE1D709
:101B40001C0E03010B6F03010B51200811E30B5115
:101B500002013F25006E000E4021016E230E00247D
:101B6000E16E000E0120E26EE66A03010B2BEBD75B
:101B70001A0E02013F25006E000E4021016E230E59
:101B80000024E16E000E0120E26E29C2E6FF2AC2A7
:101B9000E6FF0B0E3F25006E000E4021016E230E66
:101BA0000024E16E000E0120E26E200EE66E0D0EA6
:101BB00003010B6F03010B51190811E30B510201D3
:101BC0003F25006E000E4021016E230E0024E16EC1
:101BD000000E0120E26EE66A03010B2BEBD7020137
:101BE0003D5139250301596F02013E513A2103014C
:101BF0005A6F000E02013B2103015B6F000E0201D0
:101C00003C2103015C6F230E5D6F000E5E6FD0EC14
:101C100000F031EC04F01200C26AC00EC212C18C96
:101C2000C18E09C300F000360090003600900036E7
:101C300000900050C212C2804FEC04F0C284C2B4C3
:101C4000FED7080E026EC4CF00F0000E016E0250E7
:101C500005E0003600900136FF0FFAD7C35000129E
:101C6000000E0112C29012000E0E0301186F030E37
:101C7000196F09C31AF30AC31BF30BC31CF30CC37C
:101C80001DF30DC31EF3180E1F6F030E206F54ECCF
:101C900004F000C016F301C017F30050030109253A
:101CA000E16E01500A21E26EE66A16C300F017C326
:101CB00001F012001BC04DF21CC04EF21DC04FF2CD
:101CC0001EC050F273EC03F0D4EC03F018EC04F0F7
:101CD00002014D511F240301596F02014E51202072
:101CE00003015A6F000E21205B6F000E22205C6FF3
:101CF000230E5D6F000E5E6F7DEC00F0230E02017F
:101D00004F25E16E000E5021E26E29C2E6FF2AC285
:101D1000E6FF4D511F240301596F02014E5120204F
:101D200003015A6F000E21205B6F000E22205C6FB2
:101D3000230E5D6F000E5E6FD0EC00F002014D517E
:101D400025250301596F02014E51262103015A6FC7
:101D5000000E0201272103015B6F000E0201282102
:101D600003015C6F230E5D6F000E5E6FD0EC00F020
:101D700031EC04F0120014D0800E0301096F1ED064
:101D8000C00E0301096F1AD0940E0301096F16D01B
:101D9000D40E0301096F12D0800E0301096F0ED01B
:101DA00003010951010AE8E00951020AE9E0095179
:101DB000030AEAE00951040AEBE0EED703010A0541
:101DC000006E0951002600C009F300C01AF3C1ECEF
:101DD0000BF00201386B03010D6B0E6B03010D510B
:101DE0000B25E96E0E510C21EA6EEECF00F0005289
:101DF0000EE00D510B25E96E0E510C21EA6EEECF6F
:101E00001AF3C1EC0BF003010D4B0E2BE7D7010EBB
:101E10000201386F1200FAC236F2FBC237F2FAC280
:101E2000E1FFFBC2E2FFE66AFAC236F2FBC237F21A
:101E3000110EE126E76A120EE15ED4EC01F0E78AAA
:101E4000E788E786D2EC01F0E796D4EC01F0E78A68
:101E5000E788E786D2EC01F0E796E3EC01F0E3ECEB
:101E600001F0E78AE788E786D2EC01F0E796D4EC48
:101E700001F0E78AE798E786D2EC01F0E796E3EC19
:101E800001F0E78AE798E786D2EC01F0E796E78E63
:101E9000E79CE786D2EC01F0E796E3EC01F0000E58
:101EA000E76EE786D2EC01F0E796E78EE78CE78AEB
:101EB000E788E786D2EC01F0E796E3EC01F0000E4C
:101EC000E76EE786D2EC01F0E796E788E786D2EC8A
:101ED00001F0E796D4EC01F0000EE76EE786D2EC55
:101EE00001F0E796E78CE78AE786D2EC01F0E79607
:101EF000E3EC01F0010E0201386F12000301096BDF
:101F00000CEC0CF000C062F20050010F0201626F95
:101F10000301096B62C20AF314EC0CF0640E046E48
:101F200062C200F028EC0CF0300E00240201686F51
:101F3000640E046E62C200F028EC0CF008C000F0E1
:101F400000C0FAF2FAC262F20A0E046EFAC200F09F
:101F500028EC0CF0300E00240201696F0A0E046EAA
:101F6000FAC200F028EC0CF008C000F0300E00249B
:101F700002016A6F1200949A94889496C66A0201CC
:101F8000FA51C612FC51C612FB51C712FC5305E0B0
:101F9000FD51000AD8B4C78C04D00201FD53D8A467
:101FA000C78CC68A12000201FE6BFAC209F3FBC29B
:101FB0000AF3FCC20BF33AEC0CF000C059F2020138
:101FC000FE2B005203E1320EFE5DEFE3320E020102
:101FD000FE5D02E2595302E1006A12008EEC0CF041
:101FE0005AC259F35BC25AF35CC25BF35DC25CF345
:101FF000230E03015D6F000E5E6F7DEC00F00201A9
:102000002151550AD8A46BD02251AA0AD8A467D06E
:102010002350E90A08E02350EB0A03E12550900A17
:1020200002E0006A02D0010E006E00524FE1010191
:10203000ED5306E1EE5304E1EF5302E1F05309E002
:10204000E9C15AF2EAC15BF2EBC15CF2ECC15DF2AC
:102050003AD00101FD5307E1FE5305E1FF5303E1CF
:10206000020100530AE00201F9C15AF2FAC15BF21F
:10207000FBC15CF2FCC15DF226D002010D5306E10A
:102080000E5304E10F5302E1105309E009C25AF262
:102090000AC25BF20BC25CF20CC25DF214D0020108
:1020A0001D5306E11E5304E11F5302E1205309E0D2
:1020B00019C25AF21AC25BF21BC25CF21CC25DF278
:1020C00002D0006A12000201FD6B09D0010E02016C
:1020D000FD6F010E5A27000E5B235C235D23020176
:1020E000FE6B0201FD5327E15AC259F35BC25AF35A
:1020F0005CC25BF35DC25CF3230E03015D6F000EF7
:102100005E6F7DEC00F002012151550A06E122517B
:10211000AA0A03E1010E0201FD6F0201FE2B010E6E
:102120005A27000E5B235C235D23FE51400A02E127
:10213000030EFD6FD6D70201FE6B010E5A5F000E33
:102140005B5B5C5B5D5BFD51010AD8A4E4D0080ECB
:10215000046E2FC000F0000E016E045005E0003642
:1021600000900136FF0FFAD72E5000100301076FC1
:1021700001C008F3000E081307C323F208C324F2BA
:1021800030C031F2080E046E32C000F0000E016E55
:10219000045005E0003600900136FF0FFAD73150A9
:1021A00000100301056F01C006F3000E061305C3FE
:1021B00051F206C352F233C058F2080E046E3AC010
:1021C00000F0000E016E045005E00036009001366C
:1021D000FF0FFAD7395000100301036F01C004F359
:1021E000000E041303C353F204C354F233C000F0CF
:1021F000000E016E03C304F004C305F04AEC01F0C5
:10220000000E026E036E02015A5100265B5101223C
:102210005C5102225D510322030105510024020199
:10222000FF6F030106510120006F000E0220016FB5
:10223000000E0320026FFFC239F200C33AF201C35D
:102240003BF202C33CF2080E046E35C000F0000EF3
:10225000016E045005E0003600900136FF0FFAD7FA
:1022600034500012000E011200C055F201C056F2A7
:10227000050E046E045005E0003600900136FF0F95
:10228000FAD707C304F008C305F0B4EC01F000501E
:102290000201FF25326F0150030100210201336F5B
:1022A000000E030101210201346F000E030102211F
:1022B0000201356F0301055102015A25006E030129
:1022C000065102015B21016E000E5C21026E000EC0
:1022D0005D21036E00C01FF001C020F002C021F09C
:1022E00003C022F00301035100240201256F030102
:1022F000045101200201266F000E0220276F000EFC
:102300000320286F07C32BF208C32CF22C332B3386
:102310002C9F010EFE6FFEC200F0120002013F6B07
:10232000406B3D6B3E6B39C259F33AC25AF33BC224
:102330005BF33CC25CF3230E03015D6F000E5E6F26
:102340007DEC00F00301036B046B026B0201405152
:10235000241902E123513F191EE102013F6B406B3A
:102360003D4B3E2B3D5139250301596F02013E5132
:102370003A2103015A6F000E02013B2103015B6FFA
:10238000000E02013C2103015C6F230E5D6F000E05
:102390005E6F7DEC00F00301026B016B03010151E4
:1023A0000A0822E3015102013F25006E000E402180
:1023B000016E230E0024E96E000E0120EA6EEECFBE
:1023C00003F0030101510201FA25E96E000EFB2121
:1023D000EA6EEECF02F00350021802E10301022B75
:1023E00003010301012BDAD70301034B042B200E59
:1023F00002013F27000E4023030102510B0A0BE0AC
:1024000004510201561903E155510301031903E177
:102410001E0E0301026F030102510A0897E2140E17
:102420000301025D49E2200E02013F5D006E000ED5
:102430004059016E00C03FF201C040F21A0E002662
:10244000000E0122230E0024E96E000E0120EA6E28
:10245000EECF29F2EECF2AF231EC04F01C0E3F252C
:10246000006E000E4021016E230E0024E96E000E66
:102470000120EA6EEECF45F2EECF46F2EECF47F204
:10248000EECF48F2D4EC0CF00E0E02013F25006EA8
:10249000000E4021016E230E0024E96E000E012083
:1024A000EA6EEECF60F2EECF61F2EECF5EF2EECFEB
:1024B0005FF2010E006E12000201FC5309E0FAC245
:1024C00009F3FBC20AF312EC0DF0010E006E1200CC
:1024D000006A1200FAC2FEF2FBC2FFF2FEC202F074
:1024E000FFC203F00201FE4BFF2BFCC2E9FFFDC25D
:1024F000EAFFFC4BFD2BEECF00F002C0E1FF03C072
:10250000E2FF00C0E6FF02C0E9FF03C0EAFFEECF32
:1025100000F00052E3E1FAC200F0FBC201F0120049
:102520001B501F240301596F1C5020205A6F000EAE
:1025300021205B6F000E22205C6F230E5D6F000E6A
:102540005E6F7DEC00F0230E1D24E96E000E1E2050
:10255000EA6EEECFFAF2000E0201FB6FFC6FFD6F28
:10256000000EFB6FFC6FFD6FEECFFBF2000E006EF6
:102570000201FD1908E10050FC1905E1FF0EFB19ED
:1025800002E1FA51FF0A71E0FAC202F3FBC203F35F
:10259000FCC204F3FDC205F30301023702910337C5
:1025A0000437053702C3FAF203C3FBF204C3FCF29B
:1025B00005C3FDF223C204F024C205F0000E066E2E
:1025C000076E02C300F003C301F004C302F005C3A9
:1025D00003F0E9EC01F000C0FEF201C0FFF202C01E
:1025E00000F303C001F3FEC21BF0FFC21CF023C2C4
:1025F00004F024C205F0000E066E076E02C300F060
:1026000003C301F004C302F005C303F0E9EC01F0D9
:1026100008C000F009C001F00AC002F00BC003F0CE
:1026200000C01DF001C01EF00201FE511F24030175
:10263000596F0201FF51202003015A6F000E212023
:102640005B6F000E22205C6F230E5D6F000E5E6FCD
:102650007DEC00F0230E1D24E96E000E1E20EA6EB4
:10266000EECFFAF2EECFFBF281D718EC04F031ECAA
:1026700004F023C200F024C201F031C204F0000EC5
:10268000056E4AEC01F000C004F001C005F0000E38
:10269000066E076E45C200F046C201F047C202F066
:1026A00048C203F0E9EC01F008C000F009C001F0F5
:1026B0000AC002F00BC003F023C204F024C205F0EC
:1026C000000E066E076EE9EC01F000C057F20050F4
:1026D00002012D27000E2E232F23302323C204F0C6
:1026E00024C205F0000E066E076E45C200F046C219
:1026F00001F047C202F048C203F0E9EC01F008C063
:1027000000F009C001F00AC002F00BC003F000C0E5
:1027100041F201C042F202C043F203C044F212008F
:1027200002016F6B706B800E02017019006E800EDB
:10273000005C02E1080E6F5D24E2010E046E6FC2C0
:1027400000F070C201F0045005E000360090013640
:10275000FF0FFAD7710E00240201FA6F020E01205A
:10276000FB6F6FC209F30CEC0EF0FAC2E1FFFBC283
:10277000E2FF00C0E6FF01C0E6FF02016F4B702BD5
:10278000D2D71200810E0301096F020E0A6F7E0E6E
:102790000B6F2D0E0C6F000E0D6FC1C20EF3C2C277
:1027A0000FF371C210F372C211F373C212F374C249
:1027B00013F375C214F376C215F334EC0EF0020174
:1027C000C14BC22B12002DC259F32EC25AF32FC295
:1027D0005BF330C25CF3230E03015D6F000E5E6F8E
:1027E0007DEC00F00201FE6BFF6B0201FD51FF5D0D
:1027F00002E1FC51FE5D58E2230E02014125E16E2B
:10280000000E4221E26EFE51FA25E96EFF51FB21D6
:10281000EA6EEECF00F000C0E6FF010E4127000E89
:10282000422343234423000E006E441908E1005064
:10283000431905E12451421902E14151231930E1C4
:102840002DC259F32EC25AF32FC25BF330C25CF390
:10285000230E03015D6F000E5E6FD0EC00F0010EE1
:1028600002012D27000E2E232F233023416B426BB4
:10287000436B446B572B5751311903E1576B5AEC9B
:102880000EF02DC259F32EC25AF32FC25BF330C2A1
:102890005CF3230E03015D6F000E5E6F7DEC00F0B4
:1028A0000201FE4BFF2BA1D72DC259F32EC25AF3C2
:1028B0002FC25BF330C25CF3230E03015D6F000E89
:1028C0005E6FD0EC00F00201FE514527FF51462318
:1028D000000E472348233D5139250301596F02015A
:1028E0003E513A2103015A6F000E02013B210301C0
:1028F0005B6F000E02013C2103015C6F230E5D6FD4
:10290000000E5E6F7DEC00F00E0E02013F25006EA2
:10291000000E4021016E230E0024E16E000E012006
:10292000E26E60C2E6FF61C2E6FF5EC2E6FF5FC222
:10293000E6FF5EC2E6FF5FC2E6FFE66AE66A60C2E5
:10294000E6FF61C2E6FF5EC2E6FF5FC2E6FF1C0E65
:102950003F25006E000E4021016E230E0024E16E23
:10296000000E0120E26E45C2E6FF46C2E6FF47C206
:10297000E6FF48C2E6FF3D5139250301596F0201C8
:102980003E513A2103015A6F000E02013B2103011F
:102990005B6F000E02013C2103015C6F230E5D6F33
:1029A000000E5E6FD0EC00F01200FAC2FCF2FBC227
:1029B000FDF2FCC2E9FFFDC2EAFF0201FC4BFD2B68
:1029C000EECF00F00052F5E10201FA51FC5D006E1D
:1029D000FB51FD59016E010E005E000E015A1200FE
:1029E000810E0301096F020E0A6F8C0E0B6F2D0E04
:1029F0000C6F000E0D6F71C20EF372C20FF373C233
:102A000010F374C211F375C212F376C213F334ECEF
:102A10000EF0020E096F010E0A6F810E0B6F020E8F
:102A20000C6FBBEC0EF01200440E0201636F410EFE
:102A3000646F540E656F410E666F5F0E676F780EA0
:102A4000686F780E696F780E6A6F540E6B6F580E50
:102A50006C6F540E6D6F6E6B120014EC15F0530E0C
:102A60000201C76F4F0EC86F4C0EC96F410ECA6F7F
:102A7000520ECB6F200ECC6F520ECD6F450ECE6F27
:102A8000430ECF6F4F0ED06F520ED16F440ED26FE8
:102A9000450ED36F520ED46F200ED56F200ED66F19
:102AA000D76B530ED86F4F0ED96F4C0EDA6F410EA5
:102AB000DB6F520EDC6F200EDD6F520EDE6F450EA7
:102AC000DF6F430EE06F4F0EE16F520EE26F440E68
:102AD000E36F450EE46F520EE56F200EE66F200E99
:102AE000E76FE86B4E0EE96F6F0EEA6F200EEB6F2B
:102AF0004D0EEC6F650EED6F6D0EEE6F6F0EEF6F9E
:102B0000720EF06F790EF16F200EF26F200EF36FE0
:102B1000200EF46F200EF56F200EF66F200EF76F6B
:102B2000200EF86FF96B836A956A800EC16EFF0EF6
:102B3000926E080E966E850ED56EA00EF26E020E87
:102B40000C6EFF0E0B6EFF0E0A6E0C2E01D007D01E
:102B50000B2E01D003D00A2EFED7FAD7F6D7060ED9
:102B60000B6EFF0E0A6E0B2E01D003D00A2EFED77D
:102B7000FAD70A0E0A6E0A2EFED7810EFA6F0F0ED2
:102B8000FB6F0BEC0FF0010E03011A6FC1EC0BF0A1
:102B90000C0E03011A6FC1EC0BF0010E0301096F5B
:102BA000010E0A6FC70E0B6F020E0C6FBBEC0EF01E
:102BB000820E0301096F0F0E0A6F020E0B6F3AECC3
:102BC0000CF0005217E1010E0301096F010E0A6FAC
:102BD000D80E0B6F020E0C6FBBEC0EF0020E030151
:102BE000096F010E0A6FE90E0B6F020E0C6FBBEC42
:102BF0000EF0DED70201C16BC26B156A7EEC0FF0DE
:102C0000010EFA6FFB6BFC6B010EFD6FBBEC0FF05E
:102C1000820E0201FA6F0F0EFB6F020EFC6FD3ECF7
:102C20000FF0630E0201FA6F020EFB6F010EFC6FD4
:102C30008EEC11F0810E0201FA6F020EFB6F630E33
:102C4000FC6F020EFD6F6AEC12F0200E0201896F1C
:102C5000200E8A6F200E8B6F010E0301096F010E8B
:102C60000A6F810E0B6F020E0C6FBBEC0EF0820E22
:102C70000301096F0F0E0A6F020E0B6F3AEC0CF096
:102C8000005259E0165233E090EC12F090EC13F041
:102C9000C2EC13F0810E0201FA6F020EFB6FD5EC4D
:102CA00014F000C0FCF201C0FDF2810EFA6F020EBA
:102CB000FB6FE3EC13F0810E0301096F020E0A6F44
:102CC0009C0E0B6F2D0E0C6F000E0D6FC1C20EF31C
:102CD000C2C20FF334EC0EF0010E096F0C0E0A6F36
:102CE000810E0B6F020E0C6FBBEC0EF0166A020128
:102CF00090EC13F0F0EC14F0020E0C6EFF0E0B6E65
:102D0000FF0E0A6E0C2E01D007D00B2E01D003D07F
:102D10000A2EFED7FAD7F6D7060E0B6EFF0E0A6EF6
:102D20000B2E01D003D00A2EFED7FAD70A0E0A6E58
:102D30000A2EFED79CD73CD7FFD701000A006400BB
:102D4000E803102701001000000100100100080036
:102D50004000000200100080303132333435363705
:102D6000383941424344454600FF3031323334352F
:102D70003637383961626364656600FF55AA256499
:102D80002C25642C25642C25640D0A002530346420
:102D90002025303464202530346400FF253035642C
:102DA00000FFFFFFFFFFFFFFFFFFFFFFFFFFFFFF32
:020000040030CA
:0E000000FFFAFFFEFFFFFBFFFFFFFFFFFFFF0A
:00000001FF
